:0A2224000001020203030404050593
:100B2500E4F56DF56CF56BF56AC209C206C208C23B
:100B3500071221011209357E197F008E0A8F0B7568
:100B4500121975131275081975091C751019751187
:100B55005175141975157FEE54E07003020C6C7510
:100B65006E00756F808E708F71C374A99FFF7419A5
:100B75009ECF2402CF3400FEE48F698E68F567F5B9
:100B850066F565F564F563F562AF69AE68AD67ACAA
:100B950066AB65AA64A963A862C3120F775026E500
:100BA5006F2565F582E56E3564F58374CDF0E565F1
:100BB5002401F565E43564F564E43563F563E435EE
:100BC50062F56280C4E4F565F564F563F562AF69C5
:100BD500AE68AD67AC66AB65AA64A963A862C312CB
:100BE5000F775031AE64AF65E5712FF582E5703E44
:100BF500F583E0FDE56F2FF582E56E3EF583EDF0BB
:100C0500EF2401F565E43EF564E43563F563E43509
:100C150062F56280B9856E0A856F0B74002480FFCA
:100C2500741934FFFEC3E5139FF513E5129EF51203
:100C3500C3E50D9FF50DE50C9EF50CC3E50F9FF57E
:100C45000FE50E9EF50EC3E5099FF509E5089EF52E
:100C550008C3E5119FF511E5109EF510C3E5159F35
:100C6500F515E5149EF514D2E843D82090E668E022
:100C75004409F090E65CE0443DF0D2AFD288D28AD8
:100C8500C2A8C2AA43E808D2FB90E680E020E105AD
:100C9500D20A121EE890E680E054F7F0538EF8C2AF
:100CA5000930070512050BC20730092912226B50BE
:100CB50024C20912206820061690E682E030E70477
:100CC500E020E1EF90E682E030E604E020E0E41287
:0A0CD5001F1712226D12120C80C7C7
:10050B0090E6B9E070030205BC14700302063924AF
:10051B00FE70030206BC24FB70030205B6147003C5
:10052B000205B01460731460762405600302071B88
:10053B0012226F400302072790E6BBE024FE6022E5
:10054B0014603324FD601114602224067048E50A00
:10055B0090E6B3F0E50B8037E51290E6B3F0E513C8
:10056B00802DE50C90E6B3F0E50D8023E50E90E6CB
:10057B00B3F0E50F801990E6BAE0FF121F43AA060D
:10058B00A9077B01EA494B600DEE90E6B3F0EF90C3
:10059B00E6B4F00207270207201221AD020727124B
:1005AB002249020727121BE202072712219B02078F
:1005BB0027122271400302072790E6B8E0247F60E0
:1005CB001514601924027063A206E43325E0FFA220
:1005DB0008E4334F8041E490E740F0803F90E6BC65
:1005EB00E0547EFF7E00E0D394807C0040047D01CC
:1005FB0080027D00EC4EFEED4F2424F58274223EEA
:10060B00F583E493FF3395E0FEEF24A1FFEE34E690
:10061B008F82F583E0540190E740F0E4A3F090E67D
:10062B008AF090E68B7402F0020727020720122251
:10063B0073400302072790E6B8E024FE60162402FD
:10064B00600302072790E6BAE0B40105C206020771
:10065B002702072090E6BAE0705590E6BCE0547E86
:10066B00FF7E00E0D394807C0040047D0180027DFE
:10067B0000EC4EFEED4F2424F58274223EF583E40C
:10068B0093FF3395E0FEEF24A1FFEE34E68F82F566
:10069B0083E054FEF090E6BCE05480131313541F18
:1006AB00FFE0540F2F90E683F0E04420F0806D8044
:1006BB0064122275506690E6B8E024FE601924029D
:1006CB00705A90E6BAE0B40104D206804F90E6BAB5
:1006DB00E064026047803E90E6BCE0547EFF7E0003
:1006EB00E0D394807C0040047D0180027D00EC4EC1
:1006FB00FEED4F2424F58274223EF583E493FF3301
:10070B0095E0FEEF24A1FFEE34E68F82F58380089F
:10071B00120080500790E6A0E04401F090E6A0E0C4
:03072B004480F017
:01072E0022A8
:030033000218FCB4
:0418FC0053D8EF329C
:10210100758CE0758AC0E58954F04401F589758EB6
:0821110003D28CD2A9D2AF2247
:03005B0002072F6A
:10072F00C0E0C083C082C0D075D000C004C006C076
:01073F0007B2
:10074000AF91530780EF6480600302092653917FC5
:10075000300503020924E55064047070D3E53E942B
:10076000C8E53D940050030209240537E53725E02C
:100770002462F582E43428F583E53DF0A3E53EF0FC
:10078000E53725E02460F582E43428F583E0FEA314
:10079000E0FFD394C8EE9400402FEF25E0FFEE3346
:1007A000FEEF2444FFEE34FDFEE53725E02462F53C
:1007B00082E43428F583E0FCA3E0D39FEC9E40095B
:1007C000752D0175500075370002091EE550640152
:1007D0006003020884D3E53E94C8E53D94005003CD
:1007E0000209240537E53725E02462F582E4342840
:1007F000F583E53DF0A3E53EF0E53725E02460F51F
:1008000082E43428F583E0FEA3E0FFD394C8EE949D
:1008100000406EEF25E0FFEE33FEEF2444FFEE34A0
:10082000FDFEE53725E02462F582E43428F583E017
:10083000FCA3E0D39FEC9E40480551E55164027053
:100840003DE53714F534752D01E53725E0245EF5D7
:1008500082E43428F583E0FEA3E024C8F539E43EC1
:10086000F538E53725E02460F582E43428F583E0A7
:10087000FEA3E024C8F547E43EF546755000753701
:100880000002091EE55064027061C3E53E94C8E5AC
:100890003D94004048D3E53E94C8E53D94004010A7
:1008A000D3E53E9547E53D95465005752D008027DB
:1008B000D3E53E9547E53D9546400FD3E53E953956
:1008C000E53D95385004052D800DD3E53E9539E57D
:1008D0003D95384008052D753D00753E00E52D65B8
:1008E0002E7041F550F53DF53E8039E550B40534A4
:1008F000D3E53E9401E53D94004029E53725E02409
:1009000062F582E43428F583E53DF0A3E53EF00589
:1009100037052DE52DB41406755000752D00753D75
:0609200000753E00C20557
:0F092600D007D006D004D0D0D082D083D0E0321A
:101900001201000200000040181623160000010218
:1019100000010A0600020000004001000902350033
:1019200001010080FA0904000005FF00000007051E
:101930000102400000070582020002000705810243
:1019400040000007058602000200070508020002A9
:101950000009022E0001010080FA0904000004FFC2
:101960000000000705010240000007058202400058
:101970000007050202000200070581024000000482
:1019800003090410035100480059002D004300438F
:10199000004400160351004800590031003600325F
:0B19A00000300030002000200000009C
:100CDF00608028F7030A03030202030700000002E3
:100CEF00000002000A2B0B13111511110000000058
:100CFF000000003F020A0303030303070000000282
:100D0F00000002000A2B130B111511110000000037
:100D1F000000003F032D030303030307000000023D
:100D2F00000002000A2B0B13111511110000000017
:100D3F000000003F030A0A0A0A0A0A07000000021D
:100D4F00000002000A2B130B1115111100000000F7
:100D5F000000003F6024297E00000000000000001A
:100D6F000000000000000000000000000000000074
:100D7F0000000000000000000000000047297780FD
:060D8F00000009CA4E003D
:1015B70090E60174CAF090E6F574FFF0902977E0A1
:1015C70090E6F3F0902978E090E6C3F0902979E06F
:1015D70090E6C1F090297AE090E6C2F090297CE08D
:1015E70090E6C0F090297DE090E6F4F075AF0774BF
:1015F70028F59A74F7F59B759DE4E4F59EFF90E650
:101607007BE090E67CF00FBF80F490E67174FFF00A
:10161700F5B490E672E04480F043B680000000E441
:1016270090E6C4F000000090E6C5F090297EE090B7
:10163700E6C6F090297FE090E6C7F0902980E09019
:10164700E6C8F0902981E090E6C9F0902982E09001
:10165700E6CAF0902983E090E6CBF0902984E090E9
:0B166700E6CCF0902985E090E6CDF085
:011672002255
:03004300021700A1
:0300530002170091
:101700000221190002215F0002214900022131005B
:10171000021DE500021D71000216FF000222770083
:101720000222780002227900021EB70002186A0025
:1017300002227A0002227B00021D32000219AB0055
:1017400002227C000222770002227D0002227E001B
:1017500002227F00022280000222810002228200F7
:101760000222830002227700022277000222770001
:1017700002228400022285000222860002228700C3
:10178000022288000222890002228A0002228B00A3
:1017900002228C0002228D0002228E0002228F0083
:1017A0000222900002229100022292000222930063
:0817B0000222940002229500C0
:101F170090E682E030E004E020E60B90E682E030D5
:101F2700E119E030E71590E680E04401F07F147E88
:0C1F370000121CEC90E680E054FEF0224A
:1020680090E682E044C0F090E681F04387010000EA
:042078000000002242
:101EE800300A0990E680E0440AF0800790E680E036
:101EF8004408F07FDC7E05121CEC90E65D74FFF070
:0F1F080090E65FF05391EF90E680E054F7F022FF
:021F4300A907EC
:101F4500AE14AF158F828E83A3E064037017AD01C5
:101F550019ED7001228F828E83E07C002FFDEC3E0F
:091F6500FEAF0580DF7E007F0065
:011F6E002250
:101CEC008E768F7790E600E054187012E577240119
:101CFC00FFE43576C313F576EF13F577801590E690
:101D0C0000E05418FFBF100BE57725E0F577E5767A
:101D1C0033F576E5771577AE76700215764E60055D
:061D2C0012207C80EE2273
:10207C007400F58690FDA57C05A3E582458370F977
:01208C002231
:100D9500C1814228F500004228E200004228E40013
:100DA5000041280000412801004128EB00023210D3
:100DB50040C104C103014C000125004428F1000095
:100DC50000004428E700000000013C004128E6003F
:100DD50060802862000000000000000000000000A4
:100DE50000000000000000000000000000000000FE
:100DF50000000000000000000000000000000000EE
:100E050000000000000000000000000000000000DD
:100E150000000000000000000000000000000000CD
:100E250000000000000000000000000000000000BD
:100E350000000000000000000000000000000000AD
:100E4500000000000000000000000000000000009D
:100E550000000000013700015001012EFF012D00A7
:100E6500023D000001340001510002380000024635
:100E75000000014F00025700000235C350012C1934
:0B0E8500C185014100013F0001310068
:101F6F008F729028427403F0E4A3F07A287B427DAD
:101F7F00027F411220E59028427401F0A3E572F030
:0B1F8F007A287B427D027F410220E5A2
:0B220E00C2B6C2B48FB1D2B4D2B62267
:0B221900D2B6C2B48FB1D2B4D2B6224C
:10217500AE05AD077F1512220EAF0512220EAF0672
:0321850002220E25
:10218800AE05AD077F7512220EAF0512220EAF06FF
:0321980002220E12
:04204100AC05AB0738
:102045007D5FE4FF1221757D3FFF122188FEE4FDCF
:10205500AF03122219AF041222190DBD60F20EBE94
:0220650040EC4D
:012067002256
:061C9B008B5D8A5E895F8B
:101CA100E4F560F561900001120E91FC700C7D5F0E
:101CB100FF1221757D3FFF022188BCFF2DD2B67531
:101CC1006000756102C2B4AB5DAA5EA95F856182E5
:101CD100856083120E91F5B1D2B40561E5617002A0
:0A1CE1000560B482E0E560B401DBA9
:011CEB0022D6
:1014F400C2B77FC87E00121BCBD2B77FAE12220EBA
:101504007FA012220E7F7212220E7FA112220EE4FD
:10151400FF12220E7FA212220EFF12220E7FA412AD
:10152400220E7FA812220E7F3F12220E7FAD1222BE
:101534000E7F8E12220E7FB012220E7F0B12220E0D
:101544007FB112220E7F3112220E7FB312220E7F40
:10155400F012220E7F8A12220E7F6412220E7F8BDB
:1015640012220E7F7812220E7F8C12220E7F6412BA
:10157400220E7FBB12220E7F3A12220E7FBE12224F
:101584000E7F3E12220E7F8712220E7F0612220E3B
:101594007F8112220E7F9112220E7F8212220E7FF1
:1015A4005012220E7F8312220E7F7D12220E7FAFF5
:0315B40002220E02
:1009350090E600E054E74410F0000000000000904D
:10094500E61074A0F000000090E60B7401F090E64C
:100955001274E0F0000000E490E613F0000000904F
:10096500E61474E2F000000090E61574A0F00000B3
:100975000090E6D27402F090E6047480F000000066
:100985007402F00000007406F00000007408F00026
:100995000000E4F00000001215B790E6187408F0A6
:1009A50000000090E619F000000090E61AF0000043
:1009B5000090E61BF0000000E490E671F075B47F4E
:1009C50075A07F90E672F075B6FF75B1FF90E67081
:1009D500F075B2FF75B5FFC28CD2B012226690E6F3
:1009E5001074A0F000000090E611F000000090E601
:1009F5005EE04408F0000000E490E68DF0000000A1
:100A050090E65EE04404F0000000E490E7C0F0905A
:100A1500E7C4F0A3F0A3F0A3F090E7F0F090E68F21
:100A25007440F000000090E65EE04440F0000000F5
:100A35007E027F0090F800E4F0A3DFFCDEFA90E68A
:100A4500987402F0000000E490E699F00000007E42
:100A5500027F0090F800E4F0A3DFFCDEFA90E65E8A
:100A6500E04480F0000000E490E69CF00000009077
:100A7500E69DF00000007F9AFE12222E7527007574
:100A850028B47552017553907532107533B8755584
:100A95000675562C12225190E67AE054FEF0E4FDDC
:100AA5007F901221BF7F647E00121CEC7DFF7F4288
:100AB5001221BF7F647E00121CEC7D827F4E1221C5
:100AC500BF7540FF43A020E4F54490E782E540F080
:100AD50090E781E544F0122266D20575500175351F
:100AE50027753610752C05121A9D7F887E13121BEB
:100AF500CB121A9D7F887E13121BCB7FB87E0B12FB
:100B05001BCB1214F47DFFE4FF122041D2F9C2F889
:0F0B1500E4F54C90E7C0E54CF043A01053917FFE
:010B240022AE
:0E21F300EF2401FBE43EFA7D047F480220C980
:101FEF00E544C313FFC374809F9028F6F0E4940078
:101FFF009028F5F0E544D3940040067540FF43A0C8
:09200F0020E544700353A0DF2218
:10140F00E4FC9028EDE0FEA3E02400FDEC3EFC9010
:10141F002800E0FEA3E07A002400FFEA3EFEC3EDC1
:10142F009FFFEC9EFE9028E2F0A3EFF09028E5E0FE
:10143F002FF09028E4E03EF0D3EF9450EE648094C8
:10144F008050129028E2E0FAA3E0FBC394B0EA6464
:10145F0080947F501C9028E3E025E0FE9028E2E086
:10146F00339028F5F0A3CEF0E49028E4F0A3F080B9
:10147F00337C007D14AF03AE02120EE0AC06AD0755
:10148F009028E4E0FEA3E07802C333CE33CED8F940
:10149F002DFFEC3EFE7C007D0A120EF29028F5EE39
:1014AF00F0A3EFF0D39028F6E094FF9028F5E064D6
:1014BF008094804006E4F0A374FFF0C39028F5E019
:1014CF00648094805004E4F0A3F09028F5E0FEA32C
:1014DF00E0FF7C007D02120EF2C3747F9FF0E49E4A
:0414EF009028F5F05C
:0114F30022D6
:101B0F007E287FEC1221F39028EDE090E7C1F09052
:101B1F0028EEE090E7C2F09028F6E090E7C3F0904F
:101B2F0028EBE0600B43A0207540FF12140F8003D9
:101B3F00121FEF902842E540F07A287B427D017F0B
:101B4F00211220E59028427402F0A37480F07A28C5
:101B5F007B427D027F281220E5E4902842F09028F6
:101B6F00F6E0902843F07A287B427D027F280220FE
:011B7F00E580
:10120C000558E55870020557054FB53610E557B52A
:10121C00350B121B0FE4F557F5581220AC90E7C8AC
:10122C00E550F0A3E52DF0E54F652C7023E55060FB
:10123C001414600C14600924FD600504700F800008
:10124C001221E38008E4FF121F6F53A0EFE4F54F67
:10125C00200003021312754C0190E7C0E54CF0E539
:10126C00A030E7032004F87FAE12220E90F0007439
:10127C00AAF0A37411F0A374CCF0A374EEF0E49074
:10128C00E690F090E6917405F012131390F0007450
:10129C00AAF0A37411F0A374CCF0A374EEF0E49054
:1012AC00E690F090E6917405F07FAF12220EC2002A
:1012BC00E4F54C90E7C0E54CF09028E6E064017052
:1012CC002AE53C702653A0F043A0047FD07E071281
:1012DC001BCB53A0F043A00C7FD07E07121BCB532B
:1012EC00A0F043A0087FD07E078018121A9D7FB80B
:1012FC007E0B121BCB121A9D7F887E13121BCB7F89
:07130C00887E13121BCB22A7
:02226B00D3227C
:02226D00D3227A
:02226F00D32278
:101BE20090E680E030E73A00000090E6207402F0D0
:101BF200000000E490E621F000000090E624740268
:101C0200F0000000E490E625F000000090E6267463
:101C120002F0000000E490E627F0000000D201800C
:101C220016000000E490E620F000000090E6217427
:0F1C320040F0000000C20190E6BAE0F54DD32269
:10219B0090E740E54DF0E490E68AF090E68B04F092
:0221AB00D3223D
:0822490090E6BAE0F526D3226D
:1021AD0090E740E526F0E490E68AF090E68B04F0A7
:0221BD00D3222B
:02227100D32276
:02227300D32274
:02227500D32272
:10008000E4FFF572F57390E6B9E0244B60661470F6
:10009000030202A424FA70030202DC24FA700302B1
:1000A000034024F8700302038824FA70030203C695
:1000B00024FE70030204A9241F6003020507E490D4
:1000C000E68AF090E68BF090E6A0E020E1F990E679
:1000D0008BE0E4F5B390E60174CAF0D200000000B2
:1000E00090E6047480F00000007402F0000000E468
:1000F000F0020509E490E68AF090E68BF090E6A025
:10010000E020E1F990E68BE0D3943F4024E4F572DF
:1001100074402572F582E434E7F583E0FF7402252C
:1001200072F582E43428F583EFF00572E572B4408D
:10013000DF7F8A7E0012222E902802E0FF7E0012CE
:100140002237902803E075F004A4FFAEF01222409D
:10015000902807E0C394025013902823E090E6C053
:100160007005744EF08016749CF08011902823E086
:1001700090E6C07005749FF08003749DF090282570
:10018000E0F545902822E0F543902826E0F54E90D2
:100190002830E0F542A3E0FEA3E07C002400F52433
:1001A000EC3EF523902835E09028E6F0902808E012
:1001B000F53AE53A7003753A0190280DE0FEA3E0A8
:1001C0007C002400F528EC3EF527A3E0FEA3E02404
:1001D00000F553EC3EF552902809E0FEA3E0240020
:1001E000F533EC3EF532A3E0FEA3E02400F556EC37
:1001F0003EF55590283DE0FFE4FDFEFBFAF978015D
:10020000120F28A804A905AA06AB07902813E0FE40
:10021000A3E07C002400FFEC3EFEE4FDEB2FFFEAB0
:100220003EFEED39FDEC38FCC004C005C006C00739
:1002300090283EE0FFE4FCFDFEFBFA7901F8120F86
:1002400028D003D002D001D000EF2BF54BEE3AF5C9
:100250004AED39F549EC38F548902811E0FEA3E065
:100260007C002400F530EC3EF52F902837E0540F49
:10027000F53CE4FD7F901221BF902803E0FCA3E051
:10028000FDA3E0FEA3E0FF9028F1120F9B9028F160
:10029000A3E0FDA3E0FEA3E0FFE4FC9028F1120F31
:1002A0009B020509E4F57274022572F582E4342894
:1002B000F583E0FF74402572F582E434E7F583EFBF
:1002C000F00572E572B440DF000000E490E68AF0C9
:1002D00000000090E68B7440F0020509E490E68A85
:1002E000F090E68BF090E6A0E020E1F990E6BDE02A
:1002F000902842F090E6BCE0902843F0E4F572903C
:10030000E6BEE0FFE572C39F501E74402572F58281
:10031000E434E7F583E0FF74442572F582E4342881
:10032000F583EFF0057280D790E6BAE0C313FF9033
:10033000E6BEE02402FD7A287B421220E502050990
:1003400090E740740AF0A37401F0A3740CF0A37456
:1003500026F0A37407F0A374EEF0A37401F0A37465
:1003600003F0A37453F0300105E4A3F0800690E796
:100370004974FFF0000000E490E68AF0000000906D
:10038000E68B740AF002050990E6BCE09029A2F021
:100390007A297BA27D017F501220E57A297BA27DFC
:1003A000017F501220E590E6BEE0FD7AE77B407FBA
:1003B000501220C9E490E68AF000000090E6BEE00A
:1003C00090E68B020501E490E68AF090E68BF090CF
:1003D000E6A0E020E1F990E68BE0F572C29890E7A4
:1003E00040E0C394304014E534242FFFE433FEE0B2
:1003F000D39FEE6480F8748098401190E740E0F459
:100400006003020495E550600302049543A0109038
:10041000E740E0F4600AE0B4300EE52D64016008C6
:10042000D20575500402050990E740E0C3943150AD
:1004300003020509E534242FFFE433FEE0D39FEEE9
:100440006480F87480984003020509E024D1F52EF9
:10045000652D7003020509E0B40A03752E6190E76B
:1004600040E0B40B03752E6290E740E0B40C0375D6
:100470002E6390E740E0B40D03752E6490E740E0F2
:10048000B40E03752E6590E740E0B40F03752E6639
:10049000755002807490E740E06420706CE5507005
:1004A0006843A0107550058060E573C394145041F3
:1004B000E573C313FD25E02462F582E43428F58357
:1004C000E0FF74402573F582E434E7F583EFF0ED47
:1004D00025E02462F582E43428F583A3E0FF74412B
:1004E0002573F582E434E7F583EFF0057305738037
:1004F000B8000000E490E68AF000000090E68B74FB
:0A05000028F00000008002D322C39F
:01050A0022CE
:10211900C0E0C083C082D2075391EF90E65D74019D
:08212900F0D082D083D0E03237
:10214900C0E0C083C0825391EF90E65D7404F0D083
:0621590082D083D0E032C9
:10215F00C0E0C083C0825391EF90E65D7402F0D06F
:06216F0082D083D0E032B3
:101DE500C0E0C083C08285100C85110D850D8285EC
:101DF5000C83A37402F085080E85090F850F828573
:101E05000E83A37407F05391EF90E65D7410F0D044
:061E150082D083D0E03210
:10213100C0E0C083C082D2095391EF90E65D74087C
:08214100F0D082D083D0E0321F
:101D7100C0E0C083C08290E680E030E72085080C97
:101D810085090D850D82850C83A37402F085100EE3
:101D910085110F850F82850E83A37407F05391EF90
:0D1DA10090E65D7420F0D082D083D0E03257
:0116FF0032B8
:012277003234
:012278003233
:012279003232
:101EB700C0E0C083C08290E65EE054FBF000000003
:101EC70090E68F7440F00000005391EF90E65FE0DA
:101ED7004404F090E65EE04404F0D082D083D0E082
:011EE70032C8
:0D186A00C0E0C083C082C0D075D000C007B0
:1018770090E65EE054F7F090E6A1E020E1F990E70A
:1018870080E01460121460222404603614603D1452
:10189700703F752200803A90E782E0F54090E7813B
:1018A700E0F5449028EBE4F0802790E782E0902869
:1018B70000F090E781E0902801F09028EB7401F0A8
:1018C700800F90E781E024FF92048005752200D203
:1018D7000200000090E68DE4F05391EF90E65FE0A0
:0A18E7004408F090E65EE04408F0CB
:0B18F100D007D0D0D082D083D0E032EE
:01227A003231
:01227B003230
:101D3200C0E0C083C08290E65EE054BFF0000000C5
:101D420090E6987402F000000090E699E4F000003A
:101D52000090F800F0A3F05391EF90E65FE044406A
:0F1D6200F090E65EE04440F0D082D083D0E032D3
:1019AB00C0E0C083C082C0D075D000C000C001C0F1
:0B19BB0002C003C004C005C006C00746
:1019C60090E65EE0547FF090E6A6E020E1F990E62E
:1019D6009CE0FE90E69DE07C002400FFEC3EFEBE0F
:1019E600010CBF82097B017AFC7900121C9B000066
:1019F6000090E69CE4F090E69DF05391EF90E65F50
:0B1A0600E04480F090E65EE04480F0D9
:101A1100D007D006D005D004D003D002D001D00029
:091A2100D0D0D082D083D0E03295
:01227C00322F
:01227D00322E
:01227E00322D
:01227F00322C
:01228000322B
:01228100322A
:012282003229
:012283003228
:012284003227
:012285003226
:012286003225
:012287003224
:012288003223
:012289003222
:01228A003221
:01228B003220
:01228C00321F
:01228D00321E
:01228E00321D
:01228F00321C
:01229000321B
:01229100321A
:012292003219
:012293003218
:012294003217
:012295003216
:0617B8008F748C758D7624
:1017BE0053740753B0F77F0A7E00121BCBE4F57704
:1017CE00C374029577FFE574A807088002C313D887
:1017DE00FC30E00543800280035380FD7F0A7E00CB
:1017EE00121BCB4380017F0A7E00121BCB5380FE5F
:1017FE007F0A7E00121BCB0577E577C3940340C0AA
:10180E00E4F577C374099577FFE576AE75A80708FA
:10181E008005CEC313CE13D8F930E0054380028085
:10182E00035380FD7F0A7E00121BCB4380017F0A8B
:10183E007E00121BCB5380FE7F0A7E00121BCB054F
:10184E0077E577C3940A40BB43B0087F0A7E001247
:0C185E001BCB53B0F77F0A7E00021BCBAF
:09222E00AD07AC06E4FF0217B88D
:09223700AD07AC067F040217B8E4
:09224000AD07AC067F010217B8DE
:1021BF00902842EDF0EFC313FF7A287B427D010296
:0221CF0020E509
:101B800053A0F043A0087FC47E09121BCB53A0F0E2
:101B900043A00C7FC47E09121BCB53A0F043A004CA
:101BA0007FC47E09121BCB53A0F043A0067FC47EE6
:101BB00009121BCB53A0F043A0027FC47E09121B65
:0B1BC000CB53A0F043A0037FC47E09BC
:101BCB00EF7803C333CE33CED8F9FFEF4E6007EF78
:071BDB001F70F81E80F522C7
:05226600D283D28422A6
:1020AC00C2837F027E00121BCBC284D2837F027E4E
:0D20BC0000121BCBD2847F027E00021BCBE2
:1021D100E4FDFC1220AC0DBD00010CBC0EF5BD747C
:0121E100F20B
:0121E20022DA
:0722590012208D43A040227A
:0622600053A0BF022201A1
:101FC50053A0BF53A0F043A0047FD07E07121BCBC4
:101FD50053A0F043A00C7FD07E07121BCB53A0F07B
:0A1FE50043A0087FD07E07021BCB4B
:100FFC009028F1E0FCA3E0FDA3E0FEA3E0FF902825
:10100C00E7120F9BE543B40102C2B09028E6E070F2
:10101C0003122259E54560030210EA752201E47FB0
:10102C00E87E03FDFC9028E7E0F8A3E0F9A3E0FAE2
:10103C00A3E0FBC3120F7750030210D8E522640122
:10104C0060030210D87FDD7E03121CEC121B0F9084
:10105C0028E7E0FCA3E0FDA3E0FEA3E02418FFEEEC
:10106C0034FCFEED34FFFDEC34FFFC9028E7120F4E
:10107C009B9028E7E0FCA3A3A3E4FFFEFDEC78180B
:10108C00120F8890E7C4EFF09028E7A3E0FDA3A32C
:10109C00E4FFFEE4FC7810120F8890E7C5EFF090A7
:1010AC0028E7A3A3E0FEA3E4FFE4FDFC7808120FFD
:1010BC008890E7C6EFF09028E7E0FCA3E0FDA3E002
:1010CC00FEA3E0FF90E7C7EFF002102AE522B4017F
:1010DC00169028E9E0FEA3E0FF121CEC80097522B3
:1010EC0001E522640160FA9028E6E07003122260A8
:0810FC00E543B40102D2B02269
:101A2A008F798E788D778C76E4FFFEFDFCAB79AAF0
:101A3A0078A977A876D3120F774057000000E4FF01
:101A4A00FEFDE576FC7818120F8890E6CEEFF000DE
:101A5A000000E4FFFEE577FDE4FC7810120F8890A1
:101A6A00E6CFEFF0000000E4FFE578FEE4FDFC7845
:101A7A0008120F8890E6D0EFF0000000E579FF9099
:101A8A00E6D1EFF000000075BB04000000E5BB30B2
:031A9A00E7FB2245
:081DAE008C768D77AB07AA06C5
:101DB600E4FDFCC3ED9577EC95765022EA90E6D0EB
:101DC600F0000000EB90E6D1F000000075BB0500C6
:0E1DD6000000E5BB30E7FB0DBD00010C80D521
:011DE40022DC
:10201800AD07AC06000000ED25E0EC3390E6D0F00B
:10202800000000ED25E090E6D1F000000075BB044B
:09203800000000E5BB30E7FB22CB
:10131300C20253A0F043A0047FD07E07121BCB531D
:10132300A0F043A00C7FD07E07121BCB53A0F04349
:10133300A0087FD07E07121BCB9028E6E0B40107FC
:10134300E53C7003121FC51221D1754C0290E7C012
:10135300E54CF0120FFC754C0390E7C0E54CF03000
:10136300020302140EE4F574F575C3E5759528E5DB
:10137300749527500D1220AC0575E57570EC057456
:1013830080E8E542D39400400CE542FD7C00AF3396
:10139300AE32121DAED3E5249400E523940040073A
:1013A300AF24AE23122018E4F572F573C3E57395E9
:1013B30056E5729555502C121F9AE4F574F575C3D2
:1013C300E575953A7480F8657498500D1220AC0554
:1013D30075E57570EA057480E60573E57370CD05F0
:1013E3007280C9E4F574F575C3E5759553E5749595
:1013F30052500D1220AC0575E57570EC057480E84C
:0B140300AF4BAE4AAD49AC48121A2AAC
:01140E0022BB
:101F9A00000000E53325E0E5323390E6D0F000009A
:101FAA0000E53325E090E6D1F000000075BB04009F
:0B1FBA000000E5BB20E7033002F82226
:101A9D0053A0F043A0097F287E0A121BCB53A0F060
:101AAD0043A0017F287E0A121BCB53A0F043A00355
:101ABD007F287E0A121BCB53A0F043A0027F287E05
:101ACD000A121BCB53A0F043A0067F287E0A121BDF
:101ADD00CB53A0F043A0047F287E0A121BCB53A04A
:101AED00F043A00C7F287E0A121BCB53A0F043A01D
:101AFD00087F287E0A121BCBE4F52590E7CBE52560
:021B0D00F022C4
:0D220100121B8075250390E7CBE525F02228
:10208D00121B8053A0F043A001121BC753A0F043B5
:0F209D00A009121BC775250190E7CBE525F0229E
:101C41000531E531B40803E4F531E53170047F086D
:101C5100803DE531B401047F0A8034E531B40204EA
:101C61007F02802BE531B403047F038022E531B488
:101C710004047F018019E531B405047F058010E576
:101C810031B406047F048007E531B4070C7F0C12E0
:0A1C91001F6F7F2D7E00121BCB2277
:1021E300E550600B053EE53E7002053D121C4122A1
:08225100E4F51BD2E9D2AF2233
:101E1B0090E678E020E6F9C2E990E678E04480F0BD
:101E2B00EF25E090E679F090E678E030E0F990E687
:101E3B0078E04440F090E678E020E6F990E678E030
:061E4B0030E1D6D2E922CD
:101E8500A90790E678E020E6F9E51B702390E6784F
:101E9500E04480F0E925E090E679F08D16AF03A9DE
:101EA500077517018A188919E4F51A751B01D322DC
:021EB500C32246
:101E5100A90790E678E020E6F9E51B702590E67881
:101E6100E04480F0E925E0440190E679F08D16AF79
:101E710003A9077517018A188919E4F51A751B0357
:041E8100D322C32283
:03004B000211049B
:10110400C0E0C083C082C085C084C086758600C02C
:10111400D075D000C000C001C002C003C006C00723
:1011240090E678E030E206751B060211EE90E67850
:10113400E020E10CE51B64026006751B070211EE5A
:10114400E51B24FE605F14603624FE70030211DF89
:1011540024FC70030211EB240860030211EEAB17A8
:10116400AA18A919AF1A051A8F82758300120E9155
:1011740090E679F0E51A65167070751B05806B9022
:10118400E679E0AB17AA18A919AE1A8E8275830006
:10119400120EBE751B02E5166401704E90E678E0EF
:1011A4004420F08045E51624FEB51A0790E678E061
:1011B4004420F0E51614B51A0A90E678E04440F0AD
:1011C400751B0090E679E0AB17AA18A919AE1A8E20
:1011D40082758300120EBE051A800F90E678E044F3
:1011E40040F0751B008003751B005391DFD007D0BE
:1011F40006D003D002D001D000D0D0D086D084D085
:0812040085D082D083D0E032D6
:1020C900121E51E51B24FA600E146006240770F3F2
:0C20D900D322E4F51BD322E4F51BD32234
:1020E500121E85E51B24FA600E146006240770F3A2
:0C20F500D322E4F51BD322E4F51BD32218
:0300000002167372
:0C167300787FE4F6D8FD7581790216BA84
:100E9100BB010CE58229F582E5833AF583E0225016
:100EA10006E92582F8E622BBFE06E92582F8E22260
:0D0EB100E58229F582E5833AF583E493227A
:100EBE00F8BB010DE58229F582E5833AF583E8F06A
:100ECE00225006E92582C8F622BBFE05E92582C816
:020EDE00F222FE
:100EE000EF8DF0A4A8F0CF8CF0A428CE8DF0A42E26
:020EF000FE22E0
:100EF200C2D5EC30E709B2D5E4C39DFDE49CFCEE1B
:100F020030E715B2D5E4C39FFFE49EFE120FA7C3DC
:100F1200E49DFDE49CFC8003120FA730D507C3E4D7
:060F22009FFFE49EFE2289
:100F2800E88FF0A4CC8BF0A42CFCE98EF0A42CFC68
:100F38008AF0EDA42CFCEA8EF0A4CDA8F08BF0A4E6
:100F48002DCC3825F0FDE98FF0A42CCD35F0FCEB45
:100F58008EF0A4FEA9F0EB8FF0A4CFC5F02ECD390A
:0F0F6800FEE43CFCEAA42DCE35F0FDE43CFC2277
:100F7700EB9FF5F0EA9E42F0E99D42F0E89C45F0D0
:010F87002247
:100F8800E8600FECC313FCED13FDEE13FEEF13FF47
:030F9800D8F1226B
:0C0F9B00ECF0A3EDF0A3EEF0A3EFF022C9
:10167F00020B25E493A3F8E493A34003F68001F251
:10168F0008DFF48029E493A3F85407240CC8C3336C
:10169F00C4540F4420C8834004F456800146F6DF3B
:1016AF00E4800B0102040810204080900CDFE47EE0
:1016BF00019360BCA3FF543F30E509541FFEE49330
:1016CF00A360010ECF54C025E060A840B8E493A3F7
:1016DF00FAE493A3F8E493A3C8C582C8CAC583CA22
:1016EF00F0A3C8C582C8CAC583CADFE9DEE780BEDA
:010E90000061
:100FA700BC000BBE0029EF8DF084FFADF022E4CC2E
:100FB700F875F008EF2FFFEE33FEEC33FCEE9DECF7
:100FC700984005FCEE9DFE0FD5F0E9E4CEFD22ED3D
:100FD700F8F5F0EE8420D21CFEADF075F008EF2F87
:100FE700FFED33FD4007985006D5F0F222C398FD78
:050FF7000FD5F0EA2215
:00000001FF
